
 Start  Stop   Length Name               Class

 00000H 02722H 02723H _TEXT              CODE
 02724H 04791H 0206EH RTX_TEXT           CODE
 047A0H 04FE4H 00845H REG_SUPP           CODE
 04FF0H 04FF0H 00000H _FARDATA           FAR_DATA
 04FF0H 04FF4H 00005H DEMO5_DATA         FAR_DATA
 05000H 0500BH 0000CH DEMO6_DATA         FAR_DATA
 05010H 058BBH 008ACH RTX5_DATA          FAR_DATA
 058C0H 058C7H 00008H RTX6_DATA          FAR_DATA
 058D0H 058EFH 00020H RTX7_DATA          FAR_DATA
 058F0H 058F0H 00000H _FARBSS            FAR_BSS
 058F0H 058F0H 00000H _OVERLAY_          OVRINFO
 058F0H 058F0H 00000H _1STUB_            STUBSEG
 058F0H 0615DH 0086EH _DATA              DATA
 0615EH 0615FH 00002H _CVTSEG            DATA
 06160H 06165H 00006H _SCNSEG            DATA
 06170H 07113H 00FA4H T_STACK            DATA
 07114H 07114H 00000H _CONST             CONST
 07114H 07119H 00006H _INIT_             INITDATA
 0711AH 0711AH 00000H _INITEND_          INITDATA
 0711AH 0711AH 00000H _EXIT_             EXITDATA
 0711AH 0711AH 00000H _EXITEND_          EXITDATA
 0711AH 071ABH 00092H _BSS               BSS
 071ACH 071ACH 00000H _BSSEND            BSSEND
 071B0H 0722FH 00080H _STACK             STACK


Detailed map of segments

 0000:0000 0291 C=CODE   S=_TEXT          G=(none)  M=c0.ASM     ACBP=28
 0000:0291 002D C=CODE   S=_TEXT          G=(none)  M=ATEXIT     ACBP=28
 0000:02BE 003D C=CODE   S=_TEXT          G=(none)  M=DOSFATTR   ACBP=28
 0000:02FB 0093 C=CODE   S=_TEXT          G=(none)  M=EXIT       ACBP=28
 0000:038E 0000 C=CODE   S=_TEXT          G=(none)  M=FILES      ACBP=28
 0000:038E 0000 C=CODE   S=_TEXT          G=(none)  M=FILES2     ACBP=28
 0000:038E 0000 C=CODE   S=_TEXT          G=(none)  M=FMODE      ACBP=28
 0000:038E 0017 C=CODE   S=_TEXT          G=(none)  M=F_LXMUL    ACBP=28
 0000:03A5 00AE C=CODE   S=_TEXT          G=(none)  M=H_LDIV     ACBP=28
 0000:0453 0021 C=CODE   S=_TEXT          G=(none)  M=H_LLSH     ACBP=28
 0000:0474 0060 C=CODE   S=_TEXT          G=(none)  M=H_PADD     ACBP=28
 0000:04D4 004B C=CODE   S=_TEXT          G=(none)  M=IOERROR    ACBP=28
 0000:051F 0011 C=CODE   S=_TEXT          G=(none)  M=ISATTY     ACBP=28
 0000:0530 00A2 C=CODE   S=_TEXT          G=(none)  M=LONGTOA    ACBP=28
 0000:05D2 0029 C=CODE   S=_TEXT          G=(none)  M=LSEEK      ACBP=28
 0000:05FB 00B6 C=CODE   S=_TEXT          G=(none)  M=MKNAME     ACBP=28
 0000:06B1 0021 C=CODE   S=_TEXT          G=(none)  M=N_PCMP     ACBP=28
 0000:06D2 002F C=CODE   S=_TEXT          G=(none)  M=READA      ACBP=28
 0000:0701 0020 C=CODE   S=_TEXT          G=(none)  M=SEGREAD    ACBP=28
 0000:0721 00BA C=CODE   S=_TEXT          G=(none)  M=SETUPIO    ACBP=28
 0000:07DB 0018 C=CODE   S=_TEXT          G=(none)  M=UNLINK     ACBP=28
 0000:07F3 04DB C=CODE   S=_TEXT          G=(none)  M=VPRINTER   ACBP=28
 0000:0CCE 0034 C=CODE   S=_TEXT          G=(none)  M=_STPCPY    ACBP=28
 0000:0D02 001F C=CODE   S=_TEXT          G=(none)  M=CVTFAK     ACBP=28
 0000:0D21 0432 C=CODE   S=_TEXT          G=(none)  M=FARHEAP    ACBP=28
 0000:1153 0140 C=CODE   S=_TEXT          G=(none)  M=FBRK       ACBP=28
 0000:1293 00CA C=CODE   S=_TEXT          G=(none)  M=INT86      ACBP=28
 0000:135D 0029 C=CODE   S=_TEXT          G=(none)  M=IOCTL      ACBP=28
 0000:1386 0004 C=CODE   S=_TEXT          G=(none)  M=REALCVT    ACBP=28
 0000:138A 001C C=CODE   S=_TEXT          G=(none)  M=SETBLOCK   ACBP=28
 0000:13A6 001D C=CODE   S=_TEXT          G=(none)  M=CHMODA     ACBP=28
 0000:13C3 0028 C=CODE   S=_TEXT          G=(none)  M=CLOSE      ACBP=28
 0000:13EB 001E C=CODE   S=_TEXT          G=(none)  M=CLOSEA     ACBP=28
 0000:1409 0077 C=CODE   S=_TEXT          G=(none)  M=EOF        ACBP=28
 0000:1480 00B8 C=CODE   S=_TEXT          G=(none)  M=FCLOSE     ACBP=28
 0000:1538 00CD C=CODE   S=_TEXT          G=(none)  M=FFLUSH     ACBP=28
 0000:1605 009C C=CODE   S=_TEXT          G=(none)  M=FGETS      ACBP=28
 0000:16A1 0042 C=CODE   S=_TEXT          G=(none)  M=FLUSHALL   ACBP=28
 0000:16E3 020C C=CODE   S=_TEXT          G=(none)  M=FOPEN      ACBP=28
 0000:18EF 01E2 C=CODE   S=_TEXT          G=(none)  M=FSEEK      ACBP=28
 0000:1AD1 01C8 C=CODE   S=_TEXT          G=(none)  M=GETC       ACBP=28
 0000:1C99 0024 C=CODE   S=_TEXT          G=(none)  M=MEMCPY     ACBP=28
 0000:1CBD 019C C=CODE   S=_TEXT          G=(none)  M=OPEN       ACBP=28
 0000:1E59 004F C=CODE   S=_TEXT          G=(none)  M=OPENA      ACBP=28
 0000:1EA8 001B C=CODE   S=_TEXT          G=(none)  M=PRINTF     ACBP=28
 0000:1EC3 03C8 C=CODE   S=_TEXT          G=(none)  M=PUTC       ACBP=28
 0000:228B 00D1 C=CODE   S=_TEXT          G=(none)  M=READ       ACBP=28
 0000:235C 0026 C=CODE   S=_TEXT          G=(none)  M=REWIND     ACBP=28
 0000:2382 011D C=CODE   S=_TEXT          G=(none)  M=SETVBUF    ACBP=28
 0000:249F 003F C=CODE   S=_TEXT          G=(none)  M=STRCAT     ACBP=28
 0000:24DE 001F C=CODE   S=_TEXT          G=(none)  M=STRLEN     ACBP=28
 0000:24FD 0024 C=CODE   S=_TEXT          G=(none)  M=STRLWR     ACBP=28
 0000:2521 0151 C=CODE   S=_TEXT          G=(none)  M=WRITE      ACBP=28
 0000:2672 003C C=CODE   S=_TEXT          G=(none)  M=WRITEA     ACBP=28
 0000:26AE 003D C=CODE   S=_TEXT          G=(none)  M=XFCLOSE    ACBP=28
 0000:26EB 0038 C=CODE   S=_TEXT          G=(none)  M=XFFLUSH    ACBP=28
 0272:0004 0000 C=CODE   S=RTX_TEXT       G=(none)  M=RS232.ASM  ACBP=48
 0272:0004 0E18 C=CODE   S=RTX_TEXT       G=(none)  M=DEMO.C     ACBP=28
 0272:0E1C 1255 C=CODE   S=RTX_TEXT       G=(none)  M=RTX.C      ACBP=28
 0272:2072 0000 C=CODE   S=RTX_TEXT       G=(none)  M=REGS.ASM   ACBP=48
 047A:0000 03EB C=CODE   S=REG_SUPP       G=(none)  M=RS232.ASM  ACBP=68
 047A:03F0 0455 C=CODE   S=REG_SUPP       G=(none)  M=REGS.ASM   ACBP=68
 04FF:0000 0000 C=FAR_DATA S=_FARDATA       G=(none)  M=c0.ASM     ACBP=68
 04FF:0000 0005 C=FAR_DATA S=DEMO5_DATA     G=(none)  M=DEMO.C     ACBP=68
 0500:0000 000C C=FAR_DATA S=DEMO6_DATA     G=(none)  M=DEMO.C     ACBP=68
 0501:0000 08AC C=FAR_DATA S=RTX5_DATA      G=(none)  M=RTX.C      ACBP=68
 058C:0000 0008 C=FAR_DATA S=RTX6_DATA      G=(none)  M=RTX.C      ACBP=68
 058D:0000 0020 C=FAR_DATA S=RTX7_DATA      G=(none)  M=RTX.C      ACBP=68
 058F:0000 0000 C=FAR_BSS S=_FARBSS        G=(none)  M=c0.ASM     ACBP=68
 058F:0000 0000 C=OVRINFO S=_OVERLAY_      G=(none)  M=c0.ASM     ACBP=68
 058F:0000 0000 C=STUBSEG S=_1STUB_        G=(none)  M=c0.ASM     ACBP=68
 058F:0000 01A3 C=DATA   S=_DATA          G=DGROUP  M=c0.ASM     ACBP=68
 058F:01A4 00ED C=DATA   S=_DATA          G=DGROUP  M=DEMO.C     ACBP=48
 058F:0292 0307 C=DATA   S=_DATA          G=DGROUP  M=RTX.C      ACBP=48
 058F:059A 0002 C=DATA   S=_DATA          G=DGROUP  M=ATEXIT     ACBP=48
 058F:059C 0000 C=DATA   S=_DATA          G=DGROUP  M=DOSFATTR   ACBP=48
 058F:059C 000C C=DATA   S=_DATA          G=DGROUP  M=EXIT       ACBP=48
 058F:05A8 0190 C=DATA   S=_DATA          G=DGROUP  M=FILES      ACBP=48
 058F:0738 002A C=DATA   S=_DATA          G=DGROUP  M=FILES2     ACBP=48
 058F:0762 0004 C=DATA   S=_DATA          G=DGROUP  M=FMODE      ACBP=48
 058F:0766 0000 C=DATA   S=_DATA          G=DGROUP  M=F_LXMUL    ACBP=48
 058F:0766 0000 C=DATA   S=_DATA          G=DGROUP  M=H_LDIV     ACBP=48
 058F:0766 0000 C=DATA   S=_DATA          G=DGROUP  M=H_LLSH     ACBP=48
 058F:0766 0000 C=DATA   S=_DATA          G=DGROUP  M=H_PADD     ACBP=48
 058F:0766 005B C=DATA   S=_DATA          G=DGROUP  M=IOERROR    ACBP=48
 058F:07C2 0000 C=DATA   S=_DATA          G=DGROUP  M=ISATTY     ACBP=48
 058F:07C2 0000 C=DATA   S=_DATA          G=DGROUP  M=LONGTOA    ACBP=48
 058F:07C2 0000 C=DATA   S=_DATA          G=DGROUP  M=LSEEK      ACBP=48
 058F:07C2 0009 C=DATA   S=_DATA          G=DGROUP  M=MKNAME     ACBP=48
 058F:07CC 0000 C=DATA   S=_DATA          G=DGROUP  M=N_PCMP     ACBP=48
 058F:07CC 0000 C=DATA   S=_DATA          G=DGROUP  M=READA      ACBP=48
 058F:07CC 0000 C=DATA   S=_DATA          G=DGROUP  M=SEGREAD    ACBP=48
 058F:07CC 0000 C=DATA   S=_DATA          G=DGROUP  M=SETUPIO    ACBP=48
 058F:07CC 0000 C=DATA   S=_DATA          G=DGROUP  M=UNLINK     ACBP=48
 058F:07CC 0067 C=DATA   S=_DATA          G=DGROUP  M=VPRINTER   ACBP=48
 058F:0834 0000 C=DATA   S=_DATA          G=DGROUP  M=_STPCPY    ACBP=48
 058F:0834 0031 C=DATA   S=_DATA          G=DGROUP  M=CVTFAK     ACBP=48
 058F:0866 0000 C=DATA   S=_DATA          G=DGROUP  M=FARHEAP    ACBP=48
 058F:0866 0002 C=DATA   S=_DATA          G=DGROUP  M=FBRK       ACBP=48
 058F:0868 0000 C=DATA   S=_DATA          G=DGROUP  M=INT86      ACBP=48
 058F:0868 0000 C=DATA   S=_DATA          G=DGROUP  M=IOCTL      ACBP=48
 058F:0868 0000 C=DATA   S=_DATA          G=DGROUP  M=REALCVT    ACBP=48
 058F:0868 0000 C=DATA   S=_DATA          G=DGROUP  M=SETBLOCK   ACBP=48
 058F:0868 0000 C=DATA   S=_DATA          G=DGROUP  M=CHMODA     ACBP=48
 058F:0868 0000 C=DATA   S=_DATA          G=DGROUP  M=CLOSE      ACBP=48
 058F:0868 0000 C=DATA   S=_DATA          G=DGROUP  M=CLOSEA     ACBP=48
 058F:0868 0000 C=DATA   S=_DATA          G=DGROUP  M=EOF        ACBP=48
 058F:0868 0000 C=DATA   S=_DATA          G=DGROUP  M=FCLOSE     ACBP=48
 058F:0868 0000 C=DATA   S=_DATA          G=DGROUP  M=FFLUSH     ACBP=48
 058F:0868 0000 C=DATA   S=_DATA          G=DGROUP  M=FGETS      ACBP=48
 058F:0868 0000 C=DATA   S=_DATA          G=DGROUP  M=FLUSHALL   ACBP=48
 058F:0868 0000 C=DATA   S=_DATA          G=DGROUP  M=FOPEN      ACBP=48
 058F:0868 0000 C=DATA   S=_DATA          G=DGROUP  M=FSEEK      ACBP=48
 058F:0868 0000 C=DATA   S=_DATA          G=DGROUP  M=GETC       ACBP=48
 058F:0868 0000 C=DATA   S=_DATA          G=DGROUP  M=MEMCPY     ACBP=48
 058F:0868 0000 C=DATA   S=_DATA          G=DGROUP  M=OPEN       ACBP=48
 058F:0868 0000 C=DATA   S=_DATA          G=DGROUP  M=OPENA      ACBP=48
 058F:0868 0000 C=DATA   S=_DATA          G=DGROUP  M=PRINTF     ACBP=48
 058F:0868 0001 C=DATA   S=_DATA          G=DGROUP  M=PUTC       ACBP=48
 058F:086A 0000 C=DATA   S=_DATA          G=DGROUP  M=READ       ACBP=48
 058F:086A 0000 C=DATA   S=_DATA          G=DGROUP  M=REWIND     ACBP=48
 058F:086A 0004 C=DATA   S=_DATA          G=DGROUP  M=SETVBUF    ACBP=48
 058F:086E 0000 C=DATA   S=_DATA          G=DGROUP  M=STRCAT     ACBP=48
 058F:086E 0000 C=DATA   S=_DATA          G=DGROUP  M=STRLEN     ACBP=48
 058F:086E 0000 C=DATA   S=_DATA          G=DGROUP  M=STRLWR     ACBP=48
 058F:086E 0000 C=DATA   S=_DATA          G=DGROUP  M=WRITE      ACBP=48
 058F:086E 0000 C=DATA   S=_DATA          G=DGROUP  M=WRITEA     ACBP=48
 058F:086E 0000 C=DATA   S=_DATA          G=DGROUP  M=XFCLOSE    ACBP=48
 058F:086E 0000 C=DATA   S=_DATA          G=DGROUP  M=XFFLUSH    ACBP=48
 058F:086E 0000 C=DATA   S=_CVTSEG        G=DGROUP  M=c0.ASM     ACBP=48
 058F:086E 0002 C=DATA   S=_CVTSEG        G=DGROUP  M=CVTFAK     ACBP=48
 058F:0870 0000 C=DATA   S=_CVTSEG        G=DGROUP  M=REALCVT    ACBP=48
 058F:0870 0000 C=DATA   S=_SCNSEG        G=DGROUP  M=c0.ASM     ACBP=48
 058F:0870 0006 C=DATA   S=_SCNSEG        G=DGROUP  M=CVTFAK     ACBP=48
 058F:0880 0FA4 C=DATA   S=T_STACK        G=DGROUP  M=REGS.ASM   ACBP=60
 058F:1824 0000 C=CONST  S=_CONST         G=DGROUP  M=c0.ASM     ACBP=48
 058F:1824 0000 C=INITDATA S=_INIT_         G=DGROUP  M=c0.ASM     ACBP=48
 058F:1824 0006 C=INITDATA S=_INIT_         G=DGROUP  M=SETUPIO    ACBP=48
 058F:182A 0000 C=INITDATA S=_INITEND_      G=DGROUP  M=c0.ASM     ACBP=28
 058F:182A 0000 C=EXITDATA S=_EXIT_         G=DGROUP  M=c0.ASM     ACBP=48
 058F:182A 0000 C=EXITDATA S=_EXITEND_      G=DGROUP  M=c0.ASM     ACBP=28
 058F:182A 0000 C=BSS    S=_BSS           G=DGROUP  M=c0.ASM     ACBP=48
 058F:182A 0000 C=BSS    S=_BSS           G=DGROUP  M=DEMO.C     ACBP=48
 058F:182A 0000 C=BSS    S=_BSS           G=DGROUP  M=RTX.C      ACBP=48
 058F:182A 0080 C=BSS    S=_BSS           G=DGROUP  M=ATEXIT     ACBP=48
 058F:18AA 0000 C=BSS    S=_BSS           G=DGROUP  M=DOSFATTR   ACBP=48
 058F:18AA 0000 C=BSS    S=_BSS           G=DGROUP  M=IOERROR    ACBP=48
 058F:18AA 0000 C=BSS    S=_BSS           G=DGROUP  M=ISATTY     ACBP=48
 058F:18AA 0000 C=BSS    S=_BSS           G=DGROUP  M=LONGTOA    ACBP=48
 058F:18AA 0000 C=BSS    S=_BSS           G=DGROUP  M=LSEEK      ACBP=48
 058F:18AA 000D C=BSS    S=_BSS           G=DGROUP  M=MKNAME     ACBP=48
 058F:18B8 0000 C=BSS    S=_BSS           G=DGROUP  M=READA      ACBP=48
 058F:18B8 0000 C=BSS    S=_BSS           G=DGROUP  M=SEGREAD    ACBP=48
 058F:18B8 0000 C=BSS    S=_BSS           G=DGROUP  M=SETUPIO    ACBP=48
 058F:18B8 0000 C=BSS    S=_BSS           G=DGROUP  M=UNLINK     ACBP=48
 058F:18B8 0000 C=BSS    S=_BSS           G=DGROUP  M=VPRINTER   ACBP=48
 058F:18B8 0000 C=BSS    S=_BSS           G=DGROUP  M=INT86      ACBP=48
 058F:18B8 0000 C=BSS    S=_BSS           G=DGROUP  M=IOCTL      ACBP=48
 058F:18B8 0000 C=BSS    S=_BSS           G=DGROUP  M=SETBLOCK   ACBP=48
 058F:18B8 0000 C=BSS    S=_BSS           G=DGROUP  M=CHMODA     ACBP=48
 058F:18B8 0000 C=BSS    S=_BSS           G=DGROUP  M=CLOSEA     ACBP=48
 058F:18B8 0000 C=BSS    S=_BSS           G=DGROUP  M=EOF        ACBP=48
 058F:18B8 0001 C=BSS    S=_BSS           G=DGROUP  M=GETC       ACBP=48
 058F:18BA 0000 C=BSS    S=_BSS           G=DGROUP  M=MEMCPY     ACBP=48
 058F:18BA 0000 C=BSS    S=_BSS           G=DGROUP  M=OPEN       ACBP=48
 058F:18BA 0000 C=BSS    S=_BSS           G=DGROUP  M=OPENA      ACBP=48
 058F:18BA 0001 C=BSS    S=_BSS           G=DGROUP  M=PUTC       ACBP=48
 058F:18BC 0000 C=BSS    S=_BSS           G=DGROUP  M=READ       ACBP=48
 058F:18BC 0000 C=BSS    S=_BSS           G=DGROUP  M=STRCAT     ACBP=48
 058F:18BC 0000 C=BSS    S=_BSS           G=DGROUP  M=STRLEN     ACBP=48
 058F:18BC 0000 C=BSS    S=_BSS           G=DGROUP  M=STRLWR     ACBP=48
 058F:18BC 0000 C=BSS    S=_BSS           G=DGROUP  M=WRITEA     ACBP=48
 058F:18BC 0000 C=BSSEND S=_BSSEND        G=DGROUP  M=c0.ASM     ACBP=28
 071B:0000 0080 C=STACK  S=_STACK         G=(none)  M=c0.ASM     ACBP=74

  Address         Publics by Name

 0272:11C7 idle  CLEARSYSTEMEVENT
 0272:184C idle  CLEARTIMER
 0272:189A idle  CLEARTIMER_ID
 0272:0A31       COMACK
 0272:0A32 idle  COMPUTCHAR
 047A:036E       COM_ISR_EVEN
 047A:0327       COM_ISR_ODD
 047A:0577 idle  CONDENABLEINTS
 0272:19DA       COUNTDOWN_TIMERS
 047A:027B idle  CRLF_8250
 058F:0000 idle  DATASEG@
 0272:1007       DEFINEEVENTFCT
 0272:1E7B       DEFINETASK
 0000:028D idle  DGROUP@
 047A:056B       DISABLEINTS
 047A:0563       DISABLESCHED
 047A:0569       ENABLEINTS
 047A:054D       ENABLESCHED
 0272:1551       FINDTASK
 0000:03A8       F_LDIV@
 0000:03B7 idle  F_LMOD@
 0000:03AF       F_LUDIV@
 0000:03BF       F_LUMOD@
 0000:0456       F_LXLSH@
 0000:038E       F_LXMUL@
 0000:0477 idle  F_PADD@
 0000:04A6 idle  F_PSUB@
 0272:10AA idle  GETACTIVEEVENT
 047A:01EC       GETCOMBUFFER
 0272:0F61 idle  GETNEXT_QUEUEEVENT
 0272:1BB6       GETPRIORITY
 047A:0236 idle  GET_8250
 0272:1DFC       INITTASKSYSTEM
 047A:076F       INIT_INTTRAPS
 047A:03F0 idle  INSIDEDOS
 047A:0528 idle  ISCHEDULER
 0272:0FDA idle  ISNEXT_QUEUEEVENT
 047A:06F9 idle  KEYBOARDEVENTFCT
 0000:03A8 idle  LDIV@
 0000:03B7 idle  LMOD@
 0000:03AF idle  LUDIV@
 0000:03BF idle  LUMOD@
 0000:0456 idle  LXLSH@
 0000:038E idle  LXMUL@
 0272:06C0 idle  MONITOR_TASKS
 0000:03A5 idle  N_LDIV@
 0000:03B4 idle  N_LMOD@
 0000:03AC idle  N_LUDIV@
 0000:03BC idle  N_LUMOD@
 0000:0453       N_LXLSH@
 0000:0474       N_PADD@
 0000:06B1       N_PCMP@
 0000:04A3 idle  N_PSUB@
 0272:02DF idle  ONE_SECOND_INTERVAL
 0000:0477 idle  PADD@
 047A:02B6       PORT_IRQ
 0000:04A6 idle  PSUB@
 047A:025B       PUT_8250
 0272:0EDF idle  QUEUEEVENT
 0272:0E6F       QUEUEMESSAGE
 0272:09C3 idle  Q_EVENT
 047A:05FF idle  RESTORE_INTTRAPS
 0272:1104       RETURNTASK_STACKFRAME
 047A:019D       RS232_INI
 0272:112D       SAVECURRENTTASK_STACK
 047A:0418       SAVE_INITREGS
 047A:048E       SCHEDULER
 0272:1374       SCHEDULETASK
 047A:0588       SETCLOCKINTERRUPT
 0272:165C idle  SETCLOCKINTVALUE
 0272:10FA       SETKBDEVENT
 0272:1BF6       SETPRIORITY
 0272:1164 idle  SETSYSTEMEVENT
 0272:1992       SETTIMER
 0272:18A8 idle  SETTIMER_ID
 0272:042E       SHOWCOUNTS
 0272:1787 idle  SLEEPTASK
 0272:181E idle  SLEEPTILL
 0272:1D93 idle  SUSPENDTASK
 0272:00C5 idle  SYS_HAULT
 0272:09B4 idle  TASK_4
 0272:1FEA idle  TERMINATETASK
 0272:2056       TERMINATETASK_ID
 0272:122E idle  TOGGLESYSTEMEVENT
 0272:051A idle  TYPEOUT_FILE
 0272:1045 idle  WAITEVENT
 0272:10EB       WAITKBDEVENT
 0000:0276       _abort
 0501:08A0 idle  _actual_tasks
 0501:08A2 idle  _actual_timers
 0000:0291 idle  _atexit
 0000:13C3       _close
 0501:0000 idle  _Counters
 0501:08A4       _currentTask
 0272:0E5F       _disablePortIRQ
 0272:0E4E       _enablePortIRQ
 0000:1409       _eof
 058F:007F       _errno
 058F:0418 idle  _EventFunctions
 0000:0353       _exit
 0000:0E61       _farfree
 0000:0F75       _farmalloc
 0000:10D9 idle  _farrealloc
 0000:1480       _fclose
 0000:1538       _fflush
 0000:1B9F idle  _fgetc
 0000:1C8D idle  _fgetchar
 0000:1605       _fgets
 0000:16A1       _flushall
 0000:18BA       _fopen
 0000:1EDF idle  _fputc
 0000:2074 idle  _fputchar
 0000:0E61       _free
 0000:1971       _fseek
 0000:19F1 idle  _ftell
 0272:0E1C       _init_SerialPort
 0000:1293       _int86
 0000:12C4 idle  _int86x
 0000:135D       _ioctl
 0000:051F       _isatty
 0000:05D2       _lseek
 0272:0AB1       _main
 0000:0F6B       _malloc
 0000:1C99       _memcpy
 0000:1CEA       _open
 0000:1EA8       _printf
 058F:0292 idle  _queueItems
 058F:01AE idle  _queue_1
 058F:01B6 idle  _queue_2
 0000:10D2 idle  _realloc
 0000:235C       _rewind
 0000:0701       _segread
 0000:138A       _setblock
 0000:2382       _setvbuf
 0000:249F       _strcat
 0000:24DE       _strlen
 0000:24FD       _strlwr
 0501:08A8       _SystemClock
 058F:0412 idle  _SystemEvents
 058F:01BE idle  _task4_char
 0501:0100       _Tasks
 058F:01A6 idle  _Task_Counts
 0000:07DB       _unlink
 0000:1000 idle  __AHINCR
 0000:000C idle  __AHSHIFT
 058F:059A       __atexitcnt
 058F:182A       __atexittbl
 0000:11C9       __brk
 058F:008B       __brklvl
 058F:006B idle  __C0argc
 058F:006D idle  __C0argv
 058F:0071 idle  __C0environ
 0000:0374 idle  __cexit
 0000:0166       __checknull
 0000:13A6       __chmod
 0000:0153       __cleanup
 0000:13EB       __close
 0000:0000  Abs  __cvtfak
 0000:0382 idle  __c_exit
 058F:0766       __doserrno
 0000:050D       __DOSERROR
 058F:0768 idle  __dosErrorToSV
 0000:02BE       __dos_getfileattr
 0000:02DE idle  __dos_setfileattr
 058F:0093 idle  __emu
 058F:0075 idle  __envLng
 058F:0077 idle  __envseg
 058F:0079 idle  __envSize
 0000:0362       __exit
 058F:059C       __exitbuf
 058F:05A0       __exitfopen
 058F:05A4 idle  __exitopen
 0000:1B87       __fgetc
 058F:0762       __fmode
 0000:1EC3       __fputc
 0000:2088       __FPUTN
 0000:1870 idle  __GETFP
 058F:0087       __heapbase
 058F:008F       __heaptop
 058F:005B idle  __Int0Vector
 058F:005F idle  __Int4Vector
 058F:0063 idle  __Int5Vector
 058F:0067 idle  __Int6Vector
 0000:04D4       __IOERROR
 0000:0530       __LONGTOA
 0000:05FB       __MKNAME
 0000:028F idle  __MMODEL
 0000:1B9C idle  __Nfgetc
 058F:0738       __nfile
 058F:0764       __notUmask
 0000:1E59       __open
 058F:073A       __openfd
 0000:179F idle  __OPENFP
 058F:007D idle  __osmajor
 058F:007E idle  __osminor
 058F:007D idle  __osversion
 058F:007B       __psp
 0000:06D2       __read
 0000:1386       __REALCVT
 058F:086E       __RealCvtVector
 0000:01BC       __restorezero
 0000:1208       __sbrk
 058F:0870 idle  __ScanTodVector
 0000:0721       __setupio
 058F:0081 idle  __StartTime
 058F:01A4       __stklen
 0000:0CCE       __stpcpy
 058F:05A8       __streams
 0000:0167       __terminate
 0000:0658 idle  __TMPNAM
 0000:05B2       __UTOA
 058F:007D idle  __version
 0000:080B       __VPRINTER
 0000:2672       __write
 0000:26AE       __xfclose
 0000:26EB       __xfflush
 058F:0085 idle  ___brklvl
 0000:0D21 idle  ___first
 0000:0D23 idle  ___last
 0000:228B       ___read
 0000:0D25 idle  ___rover
 0000:2521       ___write

  Address         Publics by Value

 0000:0000  Abs  __cvtfak
 0000:000C idle  __AHSHIFT
 0000:0153       __cleanup
 0000:0166       __checknull
 0000:0167       __terminate
 0000:01BC       __restorezero
 0000:0276       _abort
 0000:028D idle  DGROUP@
 0000:028F idle  __MMODEL
 0000:0291 idle  _atexit
 0000:02BE       __dos_getfileattr
 0000:02DE idle  __dos_setfileattr
 0000:0353       _exit
 0000:0362       __exit
 0000:0374 idle  __cexit
 0000:0382 idle  __c_exit
 0000:038E       F_LXMUL@
 0000:038E idle  LXMUL@
 0000:03A5 idle  N_LDIV@
 0000:03A8       F_LDIV@
 0000:03A8 idle  LDIV@
 0000:03AC idle  N_LUDIV@
 0000:03AF       F_LUDIV@
 0000:03AF idle  LUDIV@
 0000:03B4 idle  N_LMOD@
 0000:03B7 idle  F_LMOD@
 0000:03B7 idle  LMOD@
 0000:03BC idle  N_LUMOD@
 0000:03BF       F_LUMOD@
 0000:03BF idle  LUMOD@
 0000:0453       N_LXLSH@
 0000:0456       F_LXLSH@
 0000:0456 idle  LXLSH@
 0000:0474       N_PADD@
 0000:0477 idle  F_PADD@
 0000:0477 idle  PADD@
 0000:04A3 idle  N_PSUB@
 0000:04A6 idle  F_PSUB@
 0000:04A6 idle  PSUB@
 0000:04D4       __IOERROR
 0000:050D       __DOSERROR
 0000:051F       _isatty
 0000:0530       __LONGTOA
 0000:05B2       __UTOA
 0000:05D2       _lseek
 0000:05FB       __MKNAME
 0000:0658 idle  __TMPNAM
 0000:06B1       N_PCMP@
 0000:06D2       __read
 0000:0701       _segread
 0000:0721       __setupio
 0000:07DB       _unlink
 0000:080B       __VPRINTER
 0000:0CCE       __stpcpy
 0000:0D21 idle  ___first
 0000:0D23 idle  ___last
 0000:0D25 idle  ___rover
 0000:0E61       _farfree
 0000:0E61       _free
 0000:0F6B       _malloc
 0000:0F75       _farmalloc
 0000:1000 idle  __AHINCR
 0000:10D2 idle  _realloc
 0000:10D9 idle  _farrealloc
 0000:11C9       __brk
 0000:1208       __sbrk
 0000:1293       _int86
 0000:12C4 idle  _int86x
 0000:135D       _ioctl
 0000:1386       __REALCVT
 0000:138A       _setblock
 0000:13A6       __chmod
 0000:13C3       _close
 0000:13EB       __close
 0000:1409       _eof
 0000:1480       _fclose
 0000:1538       _fflush
 0000:1605       _fgets
 0000:16A1       _flushall
 0000:179F idle  __OPENFP
 0000:1870 idle  __GETFP
 0000:18BA       _fopen
 0000:1971       _fseek
 0000:19F1 idle  _ftell
 0000:1B87       __fgetc
 0000:1B9C idle  __Nfgetc
 0000:1B9F idle  _fgetc
 0000:1C8D idle  _fgetchar
 0000:1C99       _memcpy
 0000:1CEA       _open
 0000:1E59       __open
 0000:1EA8       _printf
 0000:1EC3       __fputc
 0000:1EDF idle  _fputc
 0000:2074 idle  _fputchar
 0000:2088       __FPUTN
 0000:228B       ___read
 0000:235C       _rewind
 0000:2382       _setvbuf
 0000:249F       _strcat
 0000:24DE       _strlen
 0000:24FD       _strlwr
 0000:2521       ___write
 0000:2672       __write
 0000:26AE       __xfclose
 0000:26EB       __xfflush
 0272:00C5 idle  SYS_HAULT
 0272:02DF idle  ONE_SECOND_INTERVAL
 0272:042E       SHOWCOUNTS
 0272:051A idle  TYPEOUT_FILE
 0272:06C0 idle  MONITOR_TASKS
 0272:09B4 idle  TASK_4
 0272:09C3 idle  Q_EVENT
 0272:0A31       COMACK
 0272:0A32 idle  COMPUTCHAR
 0272:0AB1       _main
 0272:0E1C       _init_SerialPort
 0272:0E4E       _enablePortIRQ
 0272:0E5F       _disablePortIRQ
 0272:0E6F       QUEUEMESSAGE
 0272:0EDF idle  QUEUEEVENT
 0272:0F61 idle  GETNEXT_QUEUEEVENT
 0272:0FDA idle  ISNEXT_QUEUEEVENT
 0272:1007       DEFINEEVENTFCT
 0272:1045 idle  WAITEVENT
 0272:10AA idle  GETACTIVEEVENT
 0272:10EB       WAITKBDEVENT
 0272:10FA       SETKBDEVENT
 0272:1104       RETURNTASK_STACKFRAME
 0272:112D       SAVECURRENTTASK_STACK
 0272:1164 idle  SETSYSTEMEVENT
 0272:11C7 idle  CLEARSYSTEMEVENT
 0272:122E idle  TOGGLESYSTEMEVENT
 0272:1374       SCHEDULETASK
 0272:1551       FINDTASK
 0272:165C idle  SETCLOCKINTVALUE
 0272:1787 idle  SLEEPTASK
 0272:181E idle  SLEEPTILL
 0272:184C idle  CLEARTIMER
 0272:189A idle  CLEARTIMER_ID
 0272:18A8 idle  SETTIMER_ID
 0272:1992       SETTIMER
 0272:19DA       COUNTDOWN_TIMERS
 0272:1BB6       GETPRIORITY
 0272:1BF6       SETPRIORITY
 0272:1D93 idle  SUSPENDTASK
 0272:1DFC       INITTASKSYSTEM
 0272:1E7B       DEFINETASK
 0272:1FEA idle  TERMINATETASK
 0272:2056       TERMINATETASK_ID
 047A:019D       RS232_INI
 047A:01EC       GETCOMBUFFER
 047A:0236 idle  GET_8250
 047A:025B       PUT_8250
 047A:027B idle  CRLF_8250
 047A:02B6       PORT_IRQ
 047A:0327       COM_ISR_ODD
 047A:036E       COM_ISR_EVEN
 047A:03F0 idle  INSIDEDOS
 047A:0418       SAVE_INITREGS
 047A:048E       SCHEDULER
 047A:0528 idle  ISCHEDULER
 047A:054D       ENABLESCHED
 047A:0563       DISABLESCHED
 047A:0569       ENABLEINTS
 047A:056B       DISABLEINTS
 047A:0577 idle  CONDENABLEINTS
 047A:0588       SETCLOCKINTERRUPT
 047A:05FF idle  RESTORE_INTTRAPS
 047A:06F9 idle  KEYBOARDEVENTFCT
 047A:076F       INIT_INTTRAPS
 0501:0000 idle  _Counters
 0501:0100       _Tasks
 0501:08A0 idle  _actual_tasks
 0501:08A2 idle  _actual_timers
 0501:08A4       _currentTask
 0501:08A8       _SystemClock
 058F:0000 idle  DATASEG@
 058F:005B idle  __Int0Vector
 058F:005F idle  __Int4Vector
 058F:0063 idle  __Int5Vector
 058F:0067 idle  __Int6Vector
 058F:006B idle  __C0argc
 058F:006D idle  __C0argv
 058F:0071 idle  __C0environ
 058F:0075 idle  __envLng
 058F:0077 idle  __envseg
 058F:0079 idle  __envSize
 058F:007B       __psp
 058F:007D idle  __osversion
 058F:007D idle  __osmajor
 058F:007D idle  __version
 058F:007E idle  __osminor
 058F:007F       _errno
 058F:0081 idle  __StartTime
 058F:0085 idle  ___brklvl
 058F:0087       __heapbase
 058F:008B       __brklvl
 058F:008F       __heaptop
 058F:0093 idle  __emu
 058F:01A4       __stklen
 058F:01A6 idle  _Task_Counts
 058F:01AE idle  _queue_1
 058F:01B6 idle  _queue_2
 058F:01BE idle  _task4_char
 058F:0292 idle  _queueItems
 058F:0412 idle  _SystemEvents
 058F:0418 idle  _EventFunctions
 058F:059A       __atexitcnt
 058F:059C       __exitbuf
 058F:05A0       __exitfopen
 058F:05A4 idle  __exitopen
 058F:05A8       __streams
 058F:0738       __nfile
 058F:073A       __openfd
 058F:0762       __fmode
 058F:0764       __notUmask
 058F:0766       __doserrno
 058F:0768 idle  __dosErrorToSV
 058F:086E       __RealCvtVector
 058F:0870 idle  __ScanTodVector
 058F:182A       __atexittbl

Program entry point at 0000:0000

